:100000000C9480000C94E7060C94C0060C94A80095
:100010000C94A8000C94A8000C94A8000C94A800C0
:100020000C94A8000C9476060C94A8000C940E076F
:100030000C94A8000C94A8000C94A8000C94A800A0
:100040000C94A8000C94A8000C94A8000C94A80090
:100050000C94A8000C94A8000C94A8000C94A80080
:100060000C94A8000C94A80000404132F01110003C
:10007000002021310000000000000000000000000E
:1000800024230000000000240027002A002D000087
:10009000000000250028002B002E00005EBCE2615D
:1000A0003FDD83C29C7E20A3FD1F41009D23BE46F1
:1000B000DB65F88C11AF32CA57E9740000000023E9
:1000C00000260029002C0004040404040404040293
:1000D00002020202020303030303030505050505EB
:1000E00005050102040810204080010204081020C8
:1000F00001020408102002080104102040004307F8
:1001000011241FBECFEFD8E0DEBFCDBF11E0A0E0CD
:10011000B1E0E8E1F3E202C005900D92A03DB10725
:10012000D9F722E0A0EDB1E001C01D92A034B207E2
:10013000E1F710E0C0E8D0E004C02197FE010E9482
:100140008411CF37D107C9F70E949C070C948A11FC
:100150000C94000090913202E0913302F09134024D
:10016000292F209580FF14C0F894828182238283F6
:100170008181892B8183A3E2B0E01197F1F782811D
:10018000982B9283789487ED90E00197F1F708958A
:10019000F8948281822382838181892B8183AFEFCE
:1001A000B0E01197F1F78281982B928378948FE0D9
:1001B00090E0EBCF80913202E0913302F091340273
:1001C000F8949181982B91832281382F30952323A5
:1001D0002283A7E0B0E01197F1F7918193239183F7
:1001E000A3E2B0E01197F1F790817894EFECF0E0A2
:1001F0003197F1F7982381E009F480E00895FF92A8
:100200000F931F93CF93DF93F82E062FC8E0D0E013
:1002100011E081E09F2D912309F480E00E94AA0063
:10022000110F2197B1F7011113C0F894E091330237
:10023000F0913402918180913202809598239183CC
:10024000E0913302F0913402928189238283789481
:10025000DF91CF911F910F91FF900895809132020D
:10026000E0913302F0913402F8949181282F209587
:100270009223918378943DE743E050E0315029F197
:10028000DA011197F1F790819823C1F3F8949281E4
:10029000922392839181982B91837894ABE7B7E076
:1002A0001197F1F7F894918192239183A3E1B1E042
:1002B0001197F1F79081982381E009F080E078941C
:1002C000E3E6F6E03197F1F7089580E00895CF93E3
:1002D000DF9360E085E50E94FF00C2E1D2E060E0CC
:1002E00089910E94FF0082E0CA31D807C1F7DF91EF
:1002F000CF910895F89481E080930C020895AF9215
:10030000BF92CF92DF92EF92FF920F931F93CF9302
:10031000DF936C017B018B01040F151FEB015E0164
:10032000AE18BF08C017D10759F06991D601ED91F9
:10033000FC910190F081E02DC6010995892B79F798
:10034000C501DF91CF911F910F91FF90EF90DF904A
:10035000CF90BF90AF90089590E0FC01EE51FF4F19
:100360002491FC01E953FF4FE491EE2371F0F0E09A
:10037000EE0FFF1FE554FF4FA591B491EC91E223DE
:1003800081E090E021F480E0089580E090E008951D
:1003900090E0FC01EE51FF4F2491FC01E953FF4F27
:1003A000E491EE2389F0F0E0EE0FFF1FE157FF4FDD
:1003B000A591B4918FB7F894611107C09C91E22F79
:1003C000E095E923EC938FBF0895EC91E22BFACFEF
:1003D000CF93DF93282F30E0F901EE51FF4F449186
:1003E000F901E953FF4F9491F901E859FF4FE49166
:1003F000EE2309F446C0E051E63308F042C0F0E0D5
:10040000EC5FFD4F0C9484116C0270026C02700260
:1004100041024102410241024102410241024102C4
:1004200041024102410241023C02680241023A0299
:10043000660241024102410241024102410241027F
:1004400041024102410241024102730279027302F8
:10045000790241024102410241024102410241024C
:1004600041024102410241027D0285028B027F026C
:1004700087027F029D986D9A209180002F772093AC
:100480008000843009F04BC083E08093A000992362
:10049000D1F0892F90E0880F991FFC01ED57FF4F95
:1004A000A591B491FC01E157FF4FC591D491611121
:1004B0004CC09FB7F8948C91409584238C9388818D
:1004C000482348839FBFDF91CF9108959C986C9AF1
:1004D000209180002F7DD3CF24B52F7724BDD1CF9D
:1004E00024B52F7DFBCF2091B0002F772093B00053
:1004F000C8CF2091B0002F7DF9CF9998519A2091C3
:1005000090002F7720939000BCCF9A98529A209118
:1005100090002F7DF7CF20919000277FF3CF2AEE18
:10052000280F223020F48FEF84BF84BFB0CF8A31F0
:1005300009F0ADCF8091F00082608EBB80E880939F
:10054000F0008EB38093F000A2CF8FB7F894EC91B7
:100550004E2B4C938FBFB7CF3FB7F8948091D50106
:100560009091D601A091D701B091D8012091B2000D
:10057000B89B05C02F3F19F00196A11DB11D3FBFCB
:10058000BA2FA92F982F8827BC01CD01620F711DAA
:10059000811D911D42E0660F771F881F991F4A95A4
:1005A000D1F708958F929F92AF92BF92CF92DF9230
:1005B000EF92FF924B015C010E94AC026B017C0147
:1005C0000E94AC026C197D098E099F09683E734038
:1005D00081059105A8F321E0821A9108A108B108CC
:1005E00088EEC80E83E0D81EE11CF11C8114910432
:1005F000A104B10429F7FF90EF90DF90CF90BF9056
:10060000AF909F908F9008952FB7F8946091D1018B
:100610007091D2018091D3019091D4012FBF0895A0
:100620000895CF93DF9300D000D0CDB7DEB7FE01A1
:10063000319690E0292F280F21BD12BCF89A0000B6
:10064000000020B521939F5F9430A1F769817A81E2
:100650008B819C810F900F900F900F90DF91CF9125
:100660000895CF93DF9300D000D0CDB7DEB7498394
:100670005A836B837C83FE01319620E054E042E094
:1006800061913FB781BD92BD60BDF8945FBB4FBB28
:100690003FBF2F5F0196243099F70F900F900F9076
:1006A0000F90DF91CF910895809104019091050101
:1006B0008D31954248F580910B02882379F020E036
:1006C00030E0A9016091030270910402809105025B
:1006D000909106020E948C0F87FD16C086B386BBE0
:1006E0008091040190910501880F991F90938900D2
:1006F0008093880080916F00826080936F0080916A
:1007000081008260809381000895FC0101900020A7
:10071000E9F73197AF01481B590BBC018AE192E020
:100720000C947F018F929F92AF92BF920F931F9371
:10073000CF93DF93CDB7DEB7A1970FB6F894DEBFA6
:100740000FBECDBF19A2423008F44AE08E010F5D02
:100750001F4F842E912CB12CA12CA50194010E9435
:100760006211E62FB901CA01EA30F4F4E05DD80164
:10077000EE938D01232B242B252B79F790E080E03D
:10078000109719F0CD010E948503A1960FB6F89439
:10079000DEBF0FBECDBFDF91CF911F910F91BF90F4
:1007A000AF909F908F900895E95CE1CF0C94850302
:1007B000CF93DF93EC0160E08E810E94C80161E07D
:1007C0008E810E94C80160E08E810E94C8018BE882
:1007D00091E00197F1F7DF91CF910895CF92DF92E9
:1007E000EF92FF920F931F93CF93DF936C017C01E5
:1007F00087E0E80EF11CD0E0C0E0062F10E0B80161
:100800000C2E02C0759567950A94E2F76170F701A6
:1008100081917F010E94C8012196C430D10579F7EA
:10082000C601DF91CF911F910F91FF90EF90DF9064
:10083000CF900C94D803CF92DF92EF92FF920F9358
:100840001F93CF93DF93EC01F62E642F8C810E94CF
:10085000C8018D818F3F19F060E00E94C8010F2D03
:1008600010E08F8584FF25C06E0187E0C80ED11C83
:10087000F12CE12CB8010E2C02C0759567950A94F5
:10088000E2F76170F60181916F010E94C801FFEFEC
:10089000EF1AFF0A88E0E816F10461F7CE01DF9154
:1008A000CF911F910F91FF90EF90DF90CF900C941C
:1008B000D803B80184E0759567958A95E1F7CE0174
:1008C0000E94EE036F2DCE01DF91CF911F910F910A
:1008D000FF90EF90DF90CF900C94EE0340E0682FF4
:1008E0008AE192E00C941B0481E00E946E048BE389
:1008F0009FE10197F1F70895CF93DF93823029F4B8
:100900009091290298609093290280932D02109271
:100910002E0280E480932F0280E18093300280E5F4
:100920008093310261E080911E020E94E801809173
:100930001F028F3F19F061E00E94E80161E08091A1
:1009400020020E94E801CAE1D2E09E012A51324011
:100950008091290284FD0BC084E090E02196281745
:10096000390744F461E08E810E94E801EECF88E00F
:1009700090E0F4CF8BE39DE00197F1F760E0809188
:100980001E020E94C80160E0809120020E94C801FE
:1009900080911F028F3F19F060E00E94C801809192
:1009A000290284FD34C063E08AE192E00E94EE03F4
:1009B000CBE4D6E4CE010197F1F763E08AE192E05F
:1009C0000E94EE032197F1F763E08AE192E00E9432
:1009D000EE0383E592E00197F1F762E08AE192E0AD
:1009E0000E94EE038091290280620E946E0484E0DE
:1009F00080932A028CE00E946E040E94740482E0BC
:100A000080932B0286E0DF91CF910C946E0480627C
:100A10000E946E048BE496E40197F1F7809129021D
:100A200080620E946E0483E592E00197F1F7809165
:100A3000290280620E946E04D5CF90912D02691721
:100A400010F06FEF690FE62FF0E0E65EFD4F94893E
:100A5000890F80680C946E0441E00E941B0481E0C1
:100A600090E00895CF92DF92EF92FF926C01990F80
:100A7000EE08FF08F7FE16C041E06DE28AE192E061
:100A80000E941B0466277727CB016C197D098E090C
:100A90009F094AE00E9492030196FF90EF90DF9039
:100AA000CF9008954AE0C701B601FF90EF90DF9024
:100AB000CF900C9492034F925F926F927F928F929D
:100AC0009F92AF92BF92CF92DF92EF92FF920F93DD
:100AD0001F93CF936B017C01742EAC019B010E948C
:100AE0005D11882399F081E591E0CF911F910F91DD
:100AF000FF90EF90DF90CF90BF90AF909F908F903E
:100B00007F906F905F904F900C9485034601570142
:100B1000E894B7F82FEF3FEF4FE75FE7C501B40167
:100B20000E945D1181110DC02FEF3FEF4FE75FE78E
:100B3000C501B4010E948C0F18161CF485E591E0E4
:100B4000D4CF2FEF3FEF4FE75FE4C701B6010E941C
:100B5000EB1018161CF489E591E0C7CF2FEF3FEF9B
:100B60004FE75FECC701B6010E948C0F87FDF3CF02
:100B700020E030E0A901C701B6010E948C0F10E00F
:100B800000E087FF0CC041E06DE28AE192E00E9444
:100B90001B04F7FAF094F7F8F09401E010E0C0E0DD
:100BA00060E070E080E09FE37C1641F020E030E000
:100BB00040E251E40E94910FCF5FF6CFA70196016A
:100BC0000E94200F4B015C010E940A102B013C0186
:100BD0004AE00E949203080F191FCC23C9F1C301F8
:100BE000B2010E9439109B01AC01C501B4010E9401
:100BF0001F0F4B015C0141E06EE28AE192E00E942E
:100C00001B040F5F1F4FC15018F120E030E040E29D
:100C100051E4C501B4010E94F0102B013C010E9477
:100C20000A104B01B12CA12C4AE0C501B4010E946D
:100C30009203080F191FC501B4010E9439109B01CE
:100C4000AC01C301B2010E941F0F4B015C01DBCF5D
:100C5000C801CF911F910F91FF90EF90DF90CF903F
:100C6000BF90AF909F908F907F906F905F904F90CC
:100C7000089561E080E00E941D058DE591E00E94ED
:100C8000D60361E080E00E941D058EE691E00E949F
:100C9000D60360910D0270910E0280910F02909127
:100CA000100242E00E945B056FED8AE192E00E9433
:100CB0002C0582E791E00E94D60361E08CE00E945F
:100CC0001D056091DF017091E0018091E10190913B
:100CD000E2010E940310CB010E94320561E08FE027
:100CE0000E941D0584E791E00C94D6031F920F9299
:100CF0000FB60F9211242F933F938F939F93AF932F
:100D0000BF938091D1019091D201A091D301B09174
:100D1000D4013091D00123E0230F2D3758F50196EF
:100D2000A11DB11D2093D0018093D1019093D201D8
:100D3000A093D301B093D4018091D5019091D601B5
:100D4000A091D701B091D8010196A11DB11D80934A
:100D5000D5019093D601A093D701B093D801BF914C
:100D6000AF919F918F913F912F910F900FBE0F9058
:100D70001F90189526E8230F0296A11DB11DD2CF12
:100D80001F920F920FB60F9211242F933F934F9300
:100D90005F936F937F938F939F93AF93BF93EF93E3
:100DA000FF93E0910201F09103010995FF91EF910A
:100DB000BF91AF919F918F917F916F915F914F9173
:100DC0003F912F910F900FBE0F901F9018951F927B
:100DD0000F920FB60F9211242F933F934F935F936F
:100DE0006F937F938F939F93AF93BF93EF93FF93F3
:100DF000E0910001F09101010995FF91EF91BF9100
:100E0000AF919F918F917F916F915F914F913F91A2
:100E10002F910F900FBE0F901F9018951F920F9259
:100E20000FB60F9211242F933F934F935F936F93BD
:100E30007F938F939F93AF93BF93EF93FF93109202
:100E40006F00E1E8F0E080818C7F808361E08BE0DF
:100E50000E94C8018FE090E00197F1F760E08BE01D
:100E60000E94C801FF91EF91BF91AF919F918F9127
:100E70007F916F915F914F913F912F910F900FBE96
:100E80000F901F90189580E886BF8CE486BF60E0C5
:100E90008CE00E94E801EEEEF0E0E491A2E3B2E023
:100EA000EC93E3EDF0E0E491F0E0EE0FFF1FE5548A
:100EB000FF4F8591949112969C938E9311971B9658
:100EC0001C921B971D961C921D971C961C921C979A
:100ED0001A961C921A9719961C92199718961C929A
:100EE000189717961C92179716961C921697159698
:100EF0001C92159714961C92149713961C92EAE173
:100F0000F2E0138212828DE491E09183808381E08C
:100F100084838FEF8583168284E0878385E08087D2
:100F200086E0818787E08287138614861586168679
:100F3000178681E00C947C04CF93DF93CDB7DEB7A6
:100F4000E0970FB6F894DEBF0FBECDBF8091F200E0
:100F500080618EBB80E88093F2009EB39093F20094
:100F60008093610011E010936100789484B58260F1
:100F700084BD84B5816084BD85B5826085BD85B53D
:100F8000816085BD10928100809181008160809395
:100F90008100809181008061809381008091800038
:100FA0008260809380008FE3809387009FEF90930F
:100FB00086008091B10084608093B1008091B00080
:100FC00082608093B0008091B00081608093B00017
:100FD00080917000816080937000809191008160A9
:100FE0008093910080919100806180939100809125
:100FF00090008260809390009093960080917A0098
:10100000846080937A0080917A00826080937A0075
:1010100080917A00816080937A0080917A00806864
:1010200080937A001092C10060E082E00E94E801A3
:1010300061E082E00E94C80160E088E00E94E8016F
:1010400061E088E00E94C80160E089E00E94E80158
:1010500061E089E00E94C80160E08AE00E94E80146
:1010600061E08AE00E94C80160E083E00E94E8013C
:1010700061E083E00E94C80161E08BE00E94E8012A
:1010800084E090E00E9411036093E3017093E40117
:101090008093E5019093E60188E090E00E941103BF
:1010A0006093EF017093F0018093F1019093F2014E
:1010B0008CE090E00E9411036093F7017093F801B7
:1010C0008093F9019093FA0180E190E00E9411036E
:1010D0006093E7017093E8018093E9019093EA013E
:1010E00084E190E00E9411036093DB017093DC01C6
:1010F0008093DD019093DE0182E00E947C0460E039
:1011000080E00E941D0586E791E00E94D60361E021
:1011100080E00E941D058FE291E00E94D60360ED01
:1011200077E080E090E00E94D2020E94740489E09F
:101130000E94AC01892B09F01DC11093110260E0DF
:1011400080E00E941D0586E891E00E94D60361E0E0
:1011500080E00E941D058FE891E00E94D60389E09F
:101160000E94AC01892BD9F368EC70E080E090E03C
:101170000E94D2020E940403609307027093080247
:101180008093090290930A028AE791E0909301010B
:1011900080930001809169008C7F82608093690058
:1011A000E89A1E012AE0220E311C14E080911102FF
:1011B000882309F4B8C280910C02882309F462C024
:1011C0008091DA01882309F41FC284E1E7E0F1E0AD
:1011D000DE01559601900D928A95E1F784E1EBE1ED
:1011E000F1E0DE01119601900D928A95E1F762E03F
:1011F00070E080E090E00E94D20282E00E94AC01A8
:10120000892BE9F588E00E94AC01E090D901F12C2E
:10121000F701EE0FFF1FE15CFE4FC080D180EE0CA6
:10122000FF1CEE0CFF1CE1E0F0E0EC0FFD1FEE0EEA
:10123000FF1ED70154968D909D90AD90BC9057970E
:10124000892B09F4C2C1F601208131814281538189
:10125000C501B4010E94200F4B015C01D7014D90E4
:101260005D906D907C90A30192010E948C0F1816E6
:101270000CF4A4C1F60180829182A282B382109202
:101280000C02789489E00E94AC01892B81F5809151
:10129000DA01882309F4DBC18091D90190E0FC01D7
:1012A000EE0FFF1FE15CFE4F0190F081E02D4081C9
:1012B0005181628173810196880F991F880F991F50
:1012C0000E94310361E080E00E941D051092DA0166
:1012D00080EA91E00E94D60368EB7BE080E090E03A
:1012E0000E94D20289E00E94AC01892BD9F30E94AE
:1012F0000403C0900702D0900802E0900902F09029
:101300000A026C197D098E099F096C3271408105B2
:10131000910540F161E080E00E941D0582E691E0C8
:101320000E94D60361E080E00E941D059091DA01E1
:101330008091D901992309F4A8C1823009F4DAC156
:1013400008F094C1882309F4C8C1813009F4A9C107
:101350000E940403609307027093080280930902BD
:1013600090930A02A0E0B0E0AB2B09F41FCF0E94DB
:1013700000001CCF8091E7019091E801A091E90164
:10138000B091EA018093DF019093E001A093E10125
:10139000B093E20190E080E00E94110360930D029F
:1013A00070930E0280930F02909310021092EC0043
:1013B00010926F0010928000109281008091810045
:1013C00088608093810010928900109288008FEFCE
:1013D0009FEF90938B0080938A0011E080913F02F1
:1013E000811104C00E942E01811132C010923D0271
:1013F00010923F0210923E020E94740460E080E06E
:101400000E941D0582E991E00E94D60310923D02E0
:1014100010923F0210923E0210923C0210923B0248
:1014200010923A021092390210923802109237024A
:10143000109236021092350268EE73E080E090E080
:101440000E94D2028AE00E94AC01892B39F681C049
:1014500060E080EF0E94FF00FF24F394D12CC12CA8
:1014600001E00E94DA00E82E0E94DA0031E0E31287
:1014700036C0813009F052C0013408F4B7CFC092B1
:101480003D02C11002C010933F02809135028823B3
:1014900009F4ACCF85E392E042E152E0FA01DC01CD
:1014A0002D91CD012193B2E0EA31FB07C1F728E08D
:1014B000E0E0215009F449C0DA018D91AD018E2799
:1014C000E82FEF70F0E0E556FF4F9491E82FE2959A
:1014D000EF70F0E0E555FF4FE491E927EACFED2DFD
:1014E000F0E0E81211C080913D020817A8F4DF0176
:1014F000AE5CBD4F13968C918F2181F4E12C0930A5
:1015000010F400933E02C02EEE5CFD4F83819F2DB0
:101510009095892383830BC08013F0CFED2DF0E0ED
:10152000EE5CFD4F83818F298383EE24E3948E2D1F
:101530000E94AA000F5FFF0C19F4D394FF24F394C8
:1015400087E08D1508F08DCF97CF809119028E130B
:1015500053CF0E942E010E94670161E084E40E9443
:10156000FF000E94040360930702709308028093B7
:10157000090290930A026093FF0170930002809326
:101580000102909302028AE791E090930101809317
:101590000001809169008C7F826080936900E89AE5
:1015A00084E593E0909303018093020180916900A8
:1015B000837F886080936900E99AF3CDD6014D92CC
:1015C0005D926D927C9213975ACEA5019401F6011B
:1015D00060817181828193810E941F0F4B015C01A8
:1015E00020E030E0A9010E94EB1087FD07C0D60182
:1015F0008D929D92AD92BC92139741CEF6011082CE
:101600001182128213823BCE62E070E080E090E0B3
:101610000E94D20282E00E94AC01892B09F02FCEF9
:1016200088E00E94AC012091D901892B49F0243037
:1016300020F42F5F2093D90122CE1092D9011FCE22
:10164000222311F02150F6CF1093D90118CE81E05A
:101650008093DA016CE271E080E090E00E94D202B7
:1016600089E00E94AC01892BD9F341CE833009F483
:1016700051C0843009F06CCE6091DB017091DC01C7
:101680008091DD019091DE0114C0823079F1B8F4CF
:101690008823F9F0813009F05BCE80EB91E00E9465
:1016A000D6036091EF017091F0018091F10190916A
:1016B000F2010E940310CB010E94320549CE833013
:1016C00029F1843009F044CE8DEB91E00E94D603DD
:1016D000D3CF8CEA91E00E94D6036091E301709130
:1016E000E4018091E5019091E6010CC084EB91E06A
:1016F0000E94D6036091F7017091F8018091F90181
:101700009091FA0141E00E945B0522CE88EB91E0C6
:101710000E94D6036091E7017091E8018091E90190
:101720009091EA01C6CF89E00E94AC01892BB9F5FE
:1017300020E030E040E251E460910D0270910E0231
:1017400080910F02909110020E94F0100E940310ED
:10175000072E000C880B990B0E943B1020E030E014
:1017600040E251E40E94910FAB01BC0190E080E0A7
:101770000E94310361E080E00E941D0580EA91E053
:101780000E94D60368EB7BE080E090E00E94D202EA
:1017900089E00E94AC01892BD9F30E94390680911F
:1017A0000C028823A1F080910B02882309F494C2D3
:1017B00062E070E080E090E00E94D20282E00E944D
:1017C000AC01892B09F43BC210920C0278948AE098
:1017D0000E94AC0180930B020E940403C090070298
:1017E000D0900802E0900902F0900A026C197D097D
:1017F0008E099F09613973408105910508F49BC0EA
:101800000E942E010E94670160E08EEB0E94FF00A3
:10181000CE0101967C0188E0C82ED12C00E0BB24CB
:10182000B3940E94DA0081110B29BB0C91E0C91A14
:10183000D108B9F7D7010D937D012A163B0659F758
:1018400069817A818D81807609F09DC2687F072E3B
:10185000000C880B990B0E943B1020E030E040E820
:101860005DE30E94F0104B015C0120910302309176
:10187000040240910502509106020E941F0F6B0165
:101880007C0120E030E0A9010E94EB1018160CF05A
:1018900083C220E030E040EA51E4C701B6010E9473
:1018A0008C0F87FD84C280910601811180C2109245
:1018B00006010E942E010E94670161E084E40E94FB
:1018C000FF000E9404036093070270930802809354
:1018D000090290930A0260E080E00E941D058DE5F8
:1018E00091E00E94D60360E080E00E941D0584EC38
:1018F00091E00E94D60360910302709104028091EE
:1019000005029091060242E00E945B056FED8AE1BC
:1019100092E00E942C0588EC91E00E94D6038CECAA
:1019200091E00E94D60380910B02811104C08AEAE3
:1019300091E00E94D6030E940403C090FF01D09062
:101940000002E0900102F09002026C197D098E09FC
:101950009F09683E73408105910508F403CD0E94FC
:1019600004036093FF01709300028093010290933F
:101970000202C0900302D0900402E0900502F090B1
:10198000060280910B02882309F430C220E030E087
:10199000A901C701B6010E94EB1087FD1AC1A7017A
:1019A000960160910D0270910E0280910F0290914C
:1019B00010020E941F0F6B017C012091FB013091EE
:1019C000FC014091FD015091FE010E941F0F2091EA
:1019D000F7013091F8014091F9015091FA010E940C
:1019E000F0106093F3017093F4018093F5019093EC
:1019F000F601C092FB01D092FC01E092FD01F09251
:101A0000FE0120E030E04AE754E40E94EB10181693
:101A100064F480E090E0AAE7B4E48093F30190934B
:101A2000F401A093F501B093F60120E030E04AE71D
:101A300054EC6091F3017091F4018091F501909163
:101A4000F6010E948C0F87FF0CC080E090E0AAE7AF
:101A5000B4EC8093F3019093F401A093F501B0935B
:101A6000F6014090EF015090F0016090F10170900C
:101A7000F2018091E7019091E801A091E901B09114
:101A8000EA0189A79AA7ABA7BCA78090E301909031
:101A9000E401A090E501B090E60120E030E0A9016A
:101AA000C301B2010E94EB1018160CF096C1A301FD
:101AB0009201C701B6010E94910F2091EB01309174
:101AC000EC014091ED015091EE010E94200F2B019D
:101AD0003C0129A53AA54BA55CA560E070E088EC27
:101AE00092E40E941F0FA50194010E94910F6DA71F
:101AF0007EA78FA798AB9B01AC01C301B2010E94E6
:101B0000EB1018160CF45CC14092EB015092EC0102
:101B10006092ED017092EE01A501940169A57AA58C
:101B20008BA59CA590580E94910F2B013C01209100
:101B3000EB013091EC014091ED015091EE010E94DA
:101B4000EB10181644F44092EB015092EC016092B5
:101B5000ED017092EE012091EB013091EC0140918A
:101B6000ED015091EE01C701B6010E94200F2091B6
:101B7000F3013091F4014091F5015091F6010E947A
:101B8000200FA50194010E94F01029A53AA54BA5AC
:101B90005CA50E94200F6093DF017093E0018093A9
:101BA000E1019093E201C090DB01D090DC01E09074
:101BB000DD01F090DE01A70196010E94EB101816DE
:101BC00044F4C092DF01D092E001E092E101F09292
:101BD000E20120E030E0A9016091DF017091E001B5
:101BE0008091E1019091E2010E948C0F87FF08C073
:101BF0001092DF011092E0011092E1011092E201D7
:101C00000E9439062091DF013091E0014091E1010D
:101C10005091E20160E070E088EC92E40E941F0FB6
:101C200020E030E048EC52E40E94F0100E940310E3
:101C3000625F7E4F709305016093040193CB88E04F
:101C40000E94AC01C0900D02D0900E02E0900F02F5
:101C5000F09010022DEC3CEC4CEC5DE3892B31F163
:101C6000C701B6010E94200F6B017C0120E030E02B
:101C700040EF52E40E948C0F18164CF0C0920D02F7
:101C8000D0920E02E0920F02F09210020CC080E09F
:101C900090E0A0EFB2E480930D0290930E02A09327
:101CA0000F02B09310020E9439068ECDC701B60113
:101CB0000E941F0F6B017C0120E030E0A9010E940F
:101CC000EB1087FFDBCF10920D0210920E021092E4
:101CD0000F0210921002E7CF62E070E080E090E027
:101CE0000E94D20282E00E94AC01892B09F06CCDE7
:101CF00088E00E94AC01C090DF01D090E001E0904C
:101D0000E101F090E20120E030E040E85FE3892B60
:101D100021F1C701B6010E94200F6B017C0120E078
:101D200030E048EC52E40E948C0F18164CF0C09240
:101D3000DF01D092E001E092E101F092E201B3CF45
:101D400080E090E0A8ECB2E48093DF019093E001A2
:101D5000A093E101B093E201A6CFC701B6010E94B2
:101D60001F0F6B017C0120E030E0A9010E94EB1005
:101D700087FFDDCF1092DF011092E0011092E101A8
:101D80001092E20190CF803211F46C7F60CD8034EC
:101D900009F05DCD6E7F5BCD20E030E040EA51EC94
:101DA000C701B6010E94EB1018160CF07CCD809292
:101DB000030290920402A0920502B092060277CD2F
:101DC0008DA59EA5AFA5B8A98093EB019093EC01DA
:101DD000A093ED01B093EE019FCE1092EB01109213
:101DE000EC011092ED011092EE01B5CE8091DF0171
:101DF0009091E001A091E101B091E2018093E701AF
:101E00009093E801A093E901B093EA01C0920D021A
:101E1000D0920E02E0920F02F09210021092EB01AB
:101E20001092EC011092ED011092EE011092FB0164
:101E30001092FC011092FD011092FE01CACE505882
:101E4000BB27AA270E94370F0C94B1100E94A31041
:101E500038F00E94AA1020F039F49F3F19F426F4BC
:101E60000C94A0100EF4E095E7FB0C949A10E92F67
:101E70000E94C21058F3BA176207730784079507C8
:101E800020F079F4A6F50C94E4100EF4E0950B2EF6
:101E9000BA2FA02D0B01B90190010C01CA01A001BC
:101EA0001124FF27591B99F0593F50F4503E68F117
:101EB0001A16F040A22F232F342F4427585FF3CF58
:101EC000469537952795A795F0405395C9F77EF429
:101ED0001F16BA0B620B730B840BBAF09150A1F072
:101EE000FF0FBB1F661F771F881FC2F70EC0BA0FF8
:101EF000621F731F841F48F4879577956795B79580
:101F0000F7959E3F08F0B0CF9395880F08F099277A
:101F1000EE0F9795879508950E94761008F481E05A
:101F200008950E94A50F0C94B1100E94AA1058F0B9
:101F30000E94A31040F029F45F3F29F00C949A10FE
:101F400051110C94E5100C94A0100E94C21068F37B
:101F50009923B1F3552391F3951B550BBB27AA2762
:101F600062177307840738F09F5F5F4F220F331F9C
:101F7000441FAA1FA9F335D00E2E3AF0E0E832D064
:101F800091505040E695001CCAF72BD0FE2F29D067
:101F9000660F771F881FBB1F261737074807AB0739
:101FA000B0E809F0BB0B802DBF01FF2793585F4FAE
:101FB0003AF09E3F510578F00C949A100C94E5107D
:101FC0005F3FE4F3983ED4F3869577956795B79590
:101FD000F7959F5FC9F7880F911D9695879597F99B
:101FE0000895E1E0660F771F881FBB1F6217730714
:101FF0008407BA0720F0621B730B840BBA0BEE1F29
:1020000088F7E09508950E940A106894B1110C9425
:10201000E51008950E94CA1088F09F5798F0B92FD4
:102020009927B751B0F0E1F0660F771F881F991F0D
:102030001AF0BA95C9F714C0B13091F00E94E410BB
:10204000B1E008950C94E410672F782F8827B85FCB
:1020500039F0B93FCCF3869577956795B395D9F765
:102060003EF490958095709561957F4F8F4F9F4F6F
:102070000895E89409C097FB3EF49095809570957B
:1020800061957F4F8F4F9F4F9923A9F0F92F96E9C4
:10209000BB279395F695879577956795B795F11139
:1020A000F8CFFAF4BB0F11F460FF1BC06F5F7F4FD6
:1020B0008F4F9F4F16C0882311F096E911C07723E8
:1020C00021F09EE8872F762F05C0662371F096E8F1
:1020D000862F70E060E02AF09A95660F771F881FC0
:1020E000DAF7880F9695879597F90895990F000864
:1020F000550FAA0BE0E8FEEF16161706E807F907DA
:10210000C0F012161306E407F50798F0621B730B74
:10211000840B950B39F40A2661F0232B242B252BF5
:1021200021F408950A2609F4A140A6958FEF811D98
:10213000811D089597F99F6780E870E060E0089539
:102140009FEF80EC089500240A94161617061806CF
:102150000906089500240A941216130614060506AB
:102160000895092E0394000C11F4882352F0BB0F3C
:1021700040F4BF2B11F460FF04C06F5F7F4F8F4F9F
:102180009F4F089557FD9058440F551F59F05F3FDA
:1021900071F04795880F97FB991F61F09F3F79F089
:1021A00087950895121613061406551FF2CF46950B
:1021B000F1DF08C0161617061806991FF1CF86958D
:1021C0007105610508940895E894BB276627772771
:1021D000CB0197F908950E94761008F48FEF0895C7
:1021E0000E9403110C94B1100E94A31038F00E94B9
:1021F000AA1020F0952311F00C949A100C94A010C2
:1022000011240C94E5100E94C21070F3959FC1F345
:10221000950F50E0551F629FF001729FBB27F00D94
:10222000B11D639FAA27F00DB11DAA1F649F6627E9
:10223000B00DA11D661F829F2227B00DA11D621F38
:10224000739FB00DA11D621F839FA00D611D221FF2
:10225000749F3327A00D611D231F849F600D211DD6
:10226000822F762F6A2F11249F5750409AF0F1F059
:1022700088234AF0EE0FFF1FBB1F661F771F881FC2
:1022800091505040A9F79E3F510580F00C949A1050
:102290000C94E5105F3FE4F3983ED4F38695779570
:1022A0006795B795F795E7959F5FC1F7FE2B880F68
:1022B000911D9695879597F908950E947610880B41
:1022C000990B0895A1E21A2EAA1BBB1BFD010DC09C
:1022D000AA1FBB1FEE1FFF1FA217B307E407F507D6
:1022E00020F0A21BB30BE40BF50B661F771F881FB2
:1022F000991F1A9469F760957095809590959B0148
:10230000AC01BD01CF010895EE0FFF1F0590F491C0
:08231000E02D0994F894FFCFC1
:1023180010031003102701CDCCCC3D0000C842CDDE
:10232800CCCC3D0000803F0000803F0000C8420048
:1023380050C3470000C8420000C8420000C84244D9
:102348002E4C65646F76796920203230323100E393
:1023580001EF01F701E701DB01000000002C057F18
:10236800016E616E00696E66006F7666002020203F
:102378002020202020202020202020202000535012
:102388003D004300250054656D70526567207665F1
:102398007220342E370053455455502E2E2E004BA4
:1023A800700053656E736F72206572726F722E00C3
:1023B8002A2A2A53415645442A2A2A004B703D00AE
:1023C80054693D0054643D004F50303D004F506DFE
:1023D80061783D0050563D00432020004F500000DA
:00000001FF
